:020000040000FA
:0400000005303A2865
:08000800A000030EA100831209
:100010008B1C32288B1031181428B11C3228643004
:10002000010203183128182800001628172818285C
:1000300019281A281B281C281D281E281F283110A3
:10004000B114A810031005190314AA0DA90DA80DC9
:10005000B00B322831152A08AF002908AE00280855
:10006000AD00B11081010B11210E8300A00E200EF6
:02007000090085
:0C007400203084008001840A6030040207
:10008000031C3C281230B000A6218316FF239000E9
:10009000831283160C308505870183128501870141
:1000A000073099000030831691009F008312C830FA
:1000B00083168100831231309000003083168C004B
:1000C000831210308B00831600309B001C141A081A
:1000D0008312BC00831610309B001C141A08831274
:1000E000BD00DD2181018E018F010B118B100B10E2
:1000F0008C018B17892031199F20B30B872803109F
:1001000085190314B90DF030390203192121E521B5
:100110007A286400311808000B1D08000B11B1107B
:1001200031141230B000051D9A28321483160113C1
:100130008312080032108316011783120800311150
:100140000130B7008B132030370783169B001C1437
:100150001A088312A400A500C030A5061030370786
:1001600083169B001C141A088312A3000030370763
:1001700083169B001C141A088312A2008B17321CD2
:10018000C72822090339A200A309A409A509220846
:100190002D02031D1B2923082E02031D1B292408E1
:1001A0002F02031D1B2901303702031DDC283D18D7
:1001B000DC283D143E14AD2102303702031DE52832
:1001C000BD18E528BD143E14B32103303702031DCA
:1001D000EE283D19EE283D153E14B92104303702B2
:1001E000031DF728BD19F728BD153E14BF210530A2
:1001F0003702031D00293D1A00293D163E14C52172
:1002000006303702031D0929BD1A0929BD163E14FF
:10021000C62107303702031D12293D1B12293D1745
:100220003E14C72108303702031D1B29BD1B1B29A3
:10023000BD173E14C821B70A05303702031808005D
:10024000A2280130B600B300B400B500B7008501A4
:100250008701B1138920B30B5929031085190314A1
:10026000B90DF030390203198029B40B5929013036
:1002700037020319C921023037020319CD21033097
:1002800037020319D121043037020319D521053073
:1002900037020319D921063037020319DA21073052
:1002A00037020319DB21083037020319DC219630AD
:1002B000B400311D2A293111321C63292D0903395B
:1002C000AD00AE09AF092F1CB1132F1C2A29B11B99
:1002D0002A292E182A29B1178B1320303707BB0083
:1002E0002F08BA00932110303707BB002E08BA0040
:1002F000932100303707BB002D08BA0093218B17DC
:1003000085018701B70AB60105303702031C2A2987
:10031000DD2108003E1C08003E101030BB003D08E7
:10032000BA00932108008B133A0883161C159A0013
:100330003B089B0055309D00AA309D009C14640032
:100340009C189F291C1183128B170800FF30D000C6
:10035000D415D515D615D71508000F30D204BD1009
:100360003D11BD1108000F30D2043D103D11BD11EB
:1003700008000F30D2043D10BD10BD1108000F3031
:10038000D2043D10BD103D1108000800080008000F
:1003900008000508023A850008000508013A8500B2
:1003A00008000508203A850008000508103A850075
:1003B000080008000800080008003D08D200031DDE
:1003C00008001130BD00D20008008F080319080092
:1003D0008F01D00F732AD00A0E305205031DFF295A
:1003E000541DF529D40154160D2AD41DFA29D4011F
:1003F00054160D2A541E0D2AD401D4140D2AD41CCF
:10040000042AD40154150D2A541D092AD401D415E7
:100410000D2A541E0D2AD40154150D305205031D0A
:10042000202A551D162AD50155162E2AD51D1B2A00
:10043000D50155162E2A551E2E2AD501D5142E2A41
:10044000D51C252AD50155152E2A551D2A2AD50138
:10045000D5152E2A551E2E2AD50155150B305205BD
:10046000031D412A561D372AD60156164F2AD61D7E
:100470003C2AD60156164F2A561E4F2AD601D614AC
:100480004F2AD61C462AD60156154F2A561D4B2AEE
:10049000D601D6154F2A561E4F2AD60156150730BB
:1004A0005205031D622A571D582AD7015716702A74
:1004B000D71D5D2AD7015716702A571E702AD701FB
:1004C000D714702AD71C672AD7015715702A571DD1
:1004D0006C2AD701D715702A571E702AD7015715D5
:1004E0008A213D08D2005008D1000C305405031D6C
:1004F00085100C305505031D05100C305605031DE5
:1005000085120C305705031D051251080E02031801
:100510009D2A12305405031D851412305505031D04
:10052000051412305605031D851612305705031D9C
:100530000516FF305002031908008F08031D08003C
:10054000892051080E02031C9D2A18305405031DF2
:10055000851006305405031D851418305505031DFC
:10056000051006305505031D051418305605031DEA
:10057000851206305605031D851618305705031DD4
:0C058000051206305705031D0516080083
:084000000400030003000800A6
:02400E00CC01E3
:10420000010003000300030003000200020002009B
:1042100002000000000000000000FF00FF00FF009F
:10422000000000000000000000000000000000008E
:104230000000C000C000C000C000FF00FF00FF0081
:104240000100C300F300CF00FF00C300F300CF0064
:10425000FF00C300F300CF00FF00FF00FF00FF00DE
:10426000FF00FF00FF00FF00FF00FF00FF00FF0056
:10427000FF00FF00FF00FF00FF00FF00FF00FF0046
:10428000FF00FF00FF00FF00FF00FF00FF00FF0036
:10429000FF00FF00FF00FF00FF00FF00FF00FF0026
:1042A000FF00FF00FF00FF00FF00FF00FF00FF0016
:1042B000FF00FF00FF00FF00FF00FF00FF00FF0006
:1042C000FF00FF00FF00FF00FF00FF00FF00FF00F6
:1042D000FF00FF00FF00FF00FF00FF00FF00FF00E6
:1042E000FF00FF00FF00FF00FF00FF00FF00FF00D6
:1042F000FF00FF00FF00FF00FF00FF00FF00AA001B
:00000001FF
